S024000062696E2F6F70656E62746C5F6F6C696D65785F73746D3332703130332E737265639B
S3150800000054110020494600083546000835460008C0
S3150800001035460008354600083546000835460008C6
S3150800002035460008354600083546000835460008B6
S3150800003035460008354600083546000835460008A6
S315080000403546000835460008354600083546000896
S315080000503546000835460008354600083546000886
S315080000603546000835460008354600083546000876
S315080000703546000835460008354600083546000866
S315080000803546000835460008354600083546000856
S315080000903546000835460008354600083546000846
S315080000A03546000835460008354600083546000836
S315080000B03546000835460008354600083546000826
S315080000C03546000835460008354600083546000816
S315080000D03546000835460008354600083546000806
S315080000E035460008354600083546000835460008F6
S315080000F035460008354600083546000835460008E6
S3150800010035460008354600083546000835460008D5
S3150800011035460008354600083546000835460008C5
S3150800012035460008354600083546000835460008B5
S3150800013035460008354600083546000835460008A5
S315080001403546000835460008354600083546000895
S3150800015000B589B000230093019302930393049397
S3150800016005930693079344F2A860C0F60000694613
S3150800017002F058FD48B9009B002043B19DF80800DD
S3150800018080F01000C0F3001001E00020FFE709B07E
S315080001905DF804FB44F2A860C0F60000704700BF93
S315080001A008B540F20800C2F20000002380F82432A5
S315080001B044F2C861C0F600010A2202F091F930B98A
S315080001C040F20803C2F20003012283F8242208BD84
S315080001D038B540F20803C2F2000393F82432012B23
S315080001E005D140F20800C2F2000002F045FC4FF4C7
S315080001F08844C4F2000440252046294600F08CFEB7
S315080002000028F9D044F2A860C0F6000002F030FDDC
S3150800021038BD00BF08B540F20803C2F2000393F8E0
S315080002202432012B05D140F20800C2F2000002F088
S3150800023023FC08BD70B5064640F20803C2F2000367
S3150800024093F82432012B10D140F20801C2F20001C2
S3150800025002F0AEFD002808DA40F20800C2F20000FB
S31508000260002380F8243202F007FC317889B14FF474
S315080002708844C4F200048025204600F049FE204642
S31508000280294600F049FE0028F9D016F8011F002972
S31508000290F2D170BD00B583B00023009301934FF4EB
S315080002A08053C4F202031A6842F001021A605968C0
S315080002B00022CFF6FF020A405A601A6822F08472BA
S315080002C022F480321A601A6822F480221A605A6868
S315080002D022F4FE025A604FF41F029A601A6842F42A
S315080002E080321A604FF48053C4F2020340F2DC52A3
S315080002F0196801F4003101910099013100910199C1
S3150800030011B900999142F3D14FF48053C4F2020314
S315080003101B6813F4003F06D144F2D860C0F600000B
S31508000320732103F059FC4FF40053C4F202031A6810
S3150800033042F010021A601A6822F003021A601A685C
S3150800034042F002021A604FF48053C4F202035A685C
S315080003505A605A6842F400525A605A6842F48062F7
S315080003605A605A6822F47C125A605A6842F4E812B3
S315080003705A601A6842F080721A604FF48053C4F2C9
S3150800038002031A6812F0007FFBD04FF48053C4F2C0
S3150800039002035A6822F003025A605A6842F00202BF
S315080003A05A604FF48053C4F202035A6802F00C02F2
S315080003B0082AFAD14FF48053C4F202039A6942F02C
S315080003C009029A614FF44062C4F20102516821F0B1
S315080003D00F015160516841F008015160516821F0E0
S315080003E0F0015160516841F0B00151600022C4F239
S315080003F00102516821F4C0415160516841F48041BD
S315080004005160DA6942F00072DA61DA6942F4003260
S31508000410DA619A6942F005029A614FF40063C4F200
S3150800042001031A6822F470621A601A6842F430628C
S315080004301A601A6822F470421A601A6842F48042F6
S315080004401A6002F009FD02F015FDFCE738B5014611
S315080004504FF46050C4F2000000F040FD4FF46054C1
S31508000460C4F2000401252046294600F04BFD002869
S31508000470F9D04FF46050C4F2000000F031FDC0B26C
S3150800048038BD00BF70B503F041FE00F5FA76FF25CA
S315080004902846FFF7DBFF0446FF2803D003F036FEA5
S315080004A08642F5D8FF2C14BF0020012070BD00BF7E
S315080004B008B54FF44060C4F201004FF4805100F0D3
S315080004C0B5FCFF20FFF7C2FF08BD00BF10B54FF40B
S315080004D04060C4F201004FF4805100F0A9FCFF20EF
S315080004E0FFF7B4FFFFF7CEFF044610B9FFF7E0FFAA
S315080004F000E00124204610BD38B504460D4610F02C
S31508000500800F07D037200021FFF7F6FF01283AD8D9
S3150800051004F07F04FFF7CCFFFFF7D8FF48B344F099
S315080005204000FFF793FF280EFFF790FFC5F307403B
S31508000530FFF78CFFC5F30720FFF788FFE8B2FFF740
S3150800054085FFE4B1082C16D00120FFF77FFF0C2C9D
S3150800055002D1FF20FFF77AFF0A24FF252846FFF776
S3150800056075FF10F0800F0ED0631E13F0FF04F5D14F
S3150800057038BDFF2038BD8720FFF768FFECE79520D8
S31508000580FFF764FFE8E738BD38B505460C46FFF7C0
S3150800059079FF034620B32046FFF758FFFD2C08BF16
S315080005A001231DD0AC1C05F2022514F8020CFFF736
S315080005B04DFF14F8010CFFF749FF0234AC42F4D1A1
S315080005C0FF20FFF743FFFF20FFF740FFFF20FFF75D
S315080005D03DFF00F01F00052814BF00230123FFE795
S315080005E0184638BDF8B504460D4603F08FFD00F1F0
S315080005F06407FF263046FFF729FFFF2804D103F0DA
S3150800060085FD8742F6D818E0FE2818D10234FF2661
S315080006103046FFF71BFF04F8020C3046FFF716FFBB
S3150800062004F8010C0234023DF2D1FF20FFF70EFF59
S31508000630FF20FFF70BFF0120F8BD0020F8BD0020C2
S31508000640F8BD00BF2DE9F04389B0002840F0848149
S3150800065040F20003C2F200031B7813F0020F06D023
S3150800066040F20003C2F200031878C0B27FE1082006
S31508000670012100F0DFFB4FF48040012100F0ECFB84
S315080006804FF48058ADF800804FF010098DF80390AC
S3150800069003278DF802704FF44064C4F20104204623
S315080006A0694600F071FB2046414600F0BFFB4FF457
S315080006B02043ADF800308DF8027018238DF803300A
S315080006C02046694600F060FB4FF48046ADF80060AE
S315080006D048238DF803302046694600F055FB00256F
S315080006E0ADF808504FF48273ADF80A30ADF80C50E7
S315080006F0ADF80E50ADF810504FF40073ADF8123047
S315080007003823ADF81430ADF816500723ADF8183075
S3150800071006FA09F040F4605002A900F0AFFB06FAA9
S3150800072009F040F46050294600F0DEFB06FA09F0AD
S3150800073040F46050012100F0C3FB2046414600F01A
S3150800074075FB4FF40045ADF804508DF806708DF82A
S315080007500790204601A900F017FB2046294600F01D
S3150800076065FB0A274FF46054C4F2000402264FF0D2
S31508000770FF0801252046314600F0C4FB0028F9D0C1
S315080007802046414600F0AAFB2046294600F0BAFB5F
S315080007900028F9D0013FEDD14FF40043ADF80430FD
S315080007A003238DF8063018238DF807304FF440647C
S315080007B0C4F20104204601A900F0E6FA20464FF4E7
S315080007C0805100F035FB00200146FFF795FE012811
S315080007D040F0C48003F09AFC00F57A7408204FF4C0
S315080007E0D571FFF789FE012849D10DF11F060DF1D4
S315080007F01B05FF273846FFF729FE05F8010FB54206
S31508000800F8D19DF81E30012B40F0A8809DF81F30C6
S31508000810AA2B40F0A380A9274FF0804503F076FC69
S31508000820844205D938462946FFF766FE0028F5D1E1
S3150800083003F06CFC844240F291803A200021FFF7D5
S315080008405BFE002840F08A800DF11B04FF25284630
S31508000850FFF7FCFD04F8010FB442F8D19DF81C20FF
S3150800086002F04002D2B2002A14BF0C22042240F23F
S315080008703023C2F200031A60FFF71AFE27E0A92008
S315080008800021FFF739FE012899BF0227A92501276C
S315080008903D46002603F03AFC844205D928463146EF
S315080008A0FFF72AFE0028F5D103F030FC844255D91B
S315080008B010204FF40071FFF71FFE00284ED140F2BA
S315080008C03023C2F200031F60FFF7F2FDAFB340F218
S315080008D00003C2F200031A7802F0FE021A704FF4FF
S315080008E06055C4F200052846002100F0E9FA002404
S315080008F0ADF808404FF48273ADF80A30ADF80C40F5
S31508000900ADF80E40ADF810404FF40073ADF8123054
S315080009100823ADF81430ADF816400723ADF81830A3
S31508000920284602A900F0AAFA2846214600F0DCFA71
S315080009302846012100F0C4FA07E040F20003C2F29B
S3150800094000031A7842F001021A7040F20003C2F25C
S3150800095000031878C0B20AE0012008E040F230230C
S31508000960C2F2000300221A60FFF7A2FDE5E709B00C
S31508000970BDE8F08330B940F20003C2F200031878EC
S31508000980C0B270470120704770B50C461D46D3F1BA
S31508000990010338BF002300280CBF184643F00100A6
S315080009A000283DD140F20003C2F200031B7813F081
S315080009B0010F37D140F23023C2F200031B6813F04F
S315080009C0080F08BF5202012D0ED111201146FFF75C
S315080009D093FDF8B920464FF40071FFF703FED0F1F6
S315080009E0010538BF002515E012201146FFF784FDE2
S315080009F080B94FF4007620463146FFF7F3FD28B15B
S31508000A0004F50074013D15F0FF05F4D10C20002112
S31508000A10FFF772FDFFF74CFD281C18BF012070BDBB
S31508000A20042070BD032070BDF8B50D4617461E4656
S31508000A30D3F1010338BF002300280CBF184643F042
S31508000A40010000284DD140F20003C2F200031B78D2
S31508000A5013F0010F47D140F20003C2F200031B78DE
S31508000A6013F0040F41D140F23023C2F200031B6891
S31508000A7013F0080F08BF5702012E0DD1182039466A
S31508000A80FFF73AFD38BB2846FE21FFF77DFDD0F17A
S31508000A90010638BF00261EE013F0060F03D0972084
S31508000AA03146FFF729FD19203946FFF725FD90B98C
S31508000AB0FC2428462146FFF767FD28B105F5007591
S31508000AC0013E16F0FF06F4D10020FD21FFF75CFD7C
S31508000AD0002808BF0126FFF7EBFC301C18BF0120D1
S31508000AE0F8BD0420F8BD0320F8BD0220F8BD00BFFC
S31508000AF070B584B01446002840F03D8140F20003EA
S31508000B00C2F200031B7813F0010F18BF032040F050
S31508000B1034810E2900F21481DFE811F00F00160067
S31508000B2012015C00120112011201120112011201D6
S31508000B30C200CA00D900E800F700FFF7C7FCD0F1E9
S31508000B40010438BF002412E109200021FFF7D4FC74
S31508000B50002840F0F78068461021FFF743FD00287B
S31508000B6000F0F2809DF800309B09012B10D19DF80A
S31508000B70072002F03F02120401329DF809309DF861
S31508000B80081003EB012313449B0223600024EEE0C4
S31508000B909DF808209DF807309B0003EB92139DF8FB
S31508000BA0062002F0030203EB822201329DF805308B
S31508000BB003F00F039DF80A1003EBD1139DF80910F3
S31508000BC001F0030103EB4103073B02FA03F3236039
S31508000BD00024CCE040F23023C2F200031B6813F075
S31508000BE0040F22D08D200021FFF786FC002840F054
S31508000BF0AD80FF20FFF72AFC68461021FFF7F2FCBC
S31508000C00002800F0A5803025FF263046FFF71EFC99
S31508000C106B1E13F0FF05F8D19DF80A301B09102248
S31508000C2002FA03F323600024A1E009200021FFF75C
S31508000C3063FC002840F08E8068461021FFF7D2FC3E
S31508000C40002800F0898040F23023C2F200031B68B6
S31508000C5013F0020F12D09DF80A2002F03F029DF809
S31508000C600B30DB0903EB420201329DF80D309B097C
S31508000C70013B02FA03F32360002478E09DF80B3069
S31508000C809DF80A20C2F38402013203F003015B09CE
S31508000C9003EBC103013303FB02F32360002466E080
S31508000CA040F23023C2F200031B68137000245EE092
S31508000CB009200021FFF720FC00284FD120461021EB
S31508000CC0FFF790FCD0F1010438BF00244FE00A205A
S31508000CD00021FFF711FC002842D120461021FFF71A
S31508000CE081FCD0F1010438BF002440E03A200021FD
S31508000CF0FFF702FCB0BB0025FF263046FFF7A6FB30
S31508000D0060550135042DF8D12EE040F23023C2F2A9
S31508000D1000031B6813F0040F08BF012427D08D2099
S31508000D200021FFF7E9FB08BBFF20FFF78FFB2046F2
S31508000D304021FFF757FCD0F1010438BF002416E024
S31508000D40042414E0012412E0012410E001240EE03A
S31508000D5001240CE001240AE0012408E0012406E04D
S31508000D60012404E0012402E0002400E00124FFF746
S31508000D709FFB204601E00420FFE704B070BD00BFDA
S31508000D800020C4F2AA2070472DE9F001CB7803F0C1
S31508000D900F0513F0100F1CBF8B781D430B78F3B1AA
S31508000DA00768002301264FF00F0C06FA03F20C8899
S31508000DB0144094420FD19A000CFA02F827EA080761
S31508000DC005FA02F21743CA78282A08BF446102D0F6
S31508000DD0482A08BF04610133082BE6D107600B884F
S31508000DE0FF2B20D94768002301264FF00F0C03F18B
S31508000DF0080206FA02F20C88144094420FD19A00AF
S31508000E000CFA02F827EA080705FA02F21743CA7825
S31508000E10282A08BF4461CA78482A08BF04610133F2
S31508000E20082BE4D14760BDE8F001704701617047BF
S31508000E304161704739B14FF48053C4F202039A698D
S31508000E401043986170474FF48053C4F202039A69BD
S31508000E5022EA00009861704739B14FF48053C4F212
S31508000E600203DA691043D86170474FF48053C4F21D
S31508000E700203DA6922EA0000D861704710B40288D2
S31508000E8002F441524C880B8823438C882343CC8830
S31508000E9023430C8923434C8923438C892343CC89D8
S31508000EA0234313439BB20380838B23F400631B0401
S31508000EB01B0C83830B8A03825DF8044B704700BFC3
S31508000EC029B103889BB243F0400303807047038827
S31508000ED023F040031B041B0C038070478181704775
S31508000EE0808980B2704700BF29B103889BB243F45A
S31508000EF0005303807047038823F400531B041B0C1C
S31508000F0003807047038919420CBF002001207047EF
S31508000F10C1F3080181807047038819420CBF00207D
S31508000F200120704732B1821811F8013B00F8013BE5
S31508000F309042F9D1704700BFCA7E8B7E43EA0223EE
S31508000F400278032A01BF487D0A7D42EA002243EA65
S31508000F5002431846704700BF00F10B010023DA016F
S31508000F6042EA5303DBB210F8012B1344DBB2884282
S31508000F70F5D11846704700BF10B504460A464078B2
S31508000F8004F134010123FFF7FFFCD0BB94F83322A8
S31508000F9094F8323243EA022212B24AF65523CFF6C1
S31508000FA0FF739A422FD194F86D2094F86C301B0485
S31508000FB043EA026294F86A30134394F86B2043EAD2
S31508000FC0022222F07F4244F24613C0F254039A42A8
S31508000FD01BD094F8890094F888301B0443EA006013
S31508000FE094F88630034394F8870043EA002020F0FB
S31508000FF07F4044F24613C0F25403C01A18BF0120BA
S3150800100010BD032010BD022010BD002010BD00BF7A
S315080010102DE9F041044603791BB3056B00F134074B
S31508001020407839462A460123FFF7FEFCE0B900233B
S315080010302371636A9D421AD3E26913449D4219D209
S31508001040E678012E19D94FF00108E269154460784F
S3150800105039462A464346FFF7E7FC013E012EF4D1FE
S315080010600EE00020BDE8F0810120BDE8F0810020F7
S31508001070BDE8F0810020BDE8F0810020BDE8F081E0
S315080010800020BDE8F08100BF38B504460D46036B65
S315080010908B420CD0FFF7BCFF58B9607804F13401D5
S315080010A02A460123FFF770FC28B9256338BD0020BE
S315080010B038BD012038BD012038BD00BF08B588B14C
S315080010C003688BB1197889B1D988828891420FD182
S315080010D05878FFF74FFC00F00100002814BF0320E2
S315080010E0002008BD092008BD092008BD092008BD43
S315080010F0092008BD2DE9F041154603681C78303CE7
S31508001100092C00F2B5815A783A2A40F0B1810233A7
S31508001110036000230B60002C40F0718140F23843D5
S31508001120C2F200031C68002C00F06C810C60237866
S315080011308BB16078FFF71EFC10F0010F0BD1002D64
S3150800114000F0638100F00400C0B2002814BF0A2032
S315080011500020BDE8F081002020706070FFF772FA69
S3150800116010F0010F40F054811DB110F0040F40F04B
S31508001170528120460021FFF7FFFE012818BF0025EF
S3150800118017D194F8F631002B00F0488194F8FD2128
S3150800119094F8FC311B0443EA026294F8FA311343CB
S315080011A094F8FB5143EA052520462946FFF7E4FE55
S315080011B0FFE7032800F03581002840F0358194F8D0
S315080011C0402094F83F3043EA02231BB2B3F5007F70
S315080011D040F02D8194F84B0094F84A3053EA0020E9
S315080011E00DD194F85B2094F85A301B0443EA026246
S315080011F094F85830134394F8590043EA0020E06104
S3150800120094F84410E1704B1EDBB2012B00F21281F8
S3150800121094F84130A370002B00F00F815A1E1A4231
S3150800122040F00E8194F8466094F8452042EA06227A
S31508001230228112F00F0F40F0068194F8487094F856
S31508001240476056EA07260DD194F8577094F8566009
S31508001250360446EA076794F854603E4394F8557096
S3150800126046EA072694F843C094F8427057EA0C27D2
S3150800127000F0EC8001FB00FC07EB121161448E4282
S31508001280C0F0E780761AB6FBF3F3002B00F0E48093
S3150800129040F6F576B3428CBF022601264FF6F5785E
S315080012A0434500F2E8800233A36125622F44676252
S315080012B02944E162032E13D1002A40F0D08094F825
S315080012C0631094F86220120442EA016194F86020DF
S315080012D00A4394F8611042EA0122A2629B000EE0DA
S315080012E0002A00F0BF806744A762022E0FBF5B008A
S315080012F003225A4303F0010318BF03EB520303F218
S31508001300FF13B0EB532FC0F0B0804FF0FF332361CB
S315080013100023E360032E63D1637194F8652094F883
S31508001320643043EA02222A446261607804F1340197
S315080013300123FFF729FB002852D194F8332294F8A9
S31508001340323243EA022212B24AF65523CFF6FF7327
S315080013509A4245D194F8372094F836301B0443EA6C
S31508001360026294F83430134394F8352043EA022293
S3150800137045F25223C4F261139A4231D194F81B22E2
S3150800138094F81A321B0443EA026294F8183213439B
S3150800139094F8192243EA022247F27223C6F241134D
S315080013A09A421DD194F8232294F822321B0443EA68
S315080013B0026294F82032134394F8212243EA022366
S315080013C0E36094F81F2294F81E321B0443EA026273
S315080013D094F81C32134394F81D2243EA022323612E
S315080013E0267040F23443C2F200031A88013292B2E0
S315080013F01A80E280002020632071BDE8F0810B206E
S31508001400BDE8F0810C20BDE8F0810020BDE8F08140
S315080014100320BDE8F0810A20BDE8F0810D20BDE873
S31508001420F0810120BDE8F0810D20BDE8F0810D2096
S31508001430BDE8F0810D20BDE8F0810D20BDE8F08102
S315080014400D20BDE8F0810D20BDE8F0810D20BDE836
S31508001450F0810D20BDE8F0810D20BDE8F0810D205A
S31508001460BDE8F0810D20BDE8F0810D20BDE8F081D2
S3150800147000230B6052E60233A36125622F4467629C
S315080014802944E162032617E72DE9F0410D4601F1EB
S3150800149009020369002B5ED0416991F80C800B782C
S315080014A0202B1BD00E46002408F00807FFB203E0E5
S315080014B016F8013F202B11D0052B08BFE52347B1AD
S315080014C0A3F1410C5FFA8CFCBCF1190F9CBF2033C9
S315080014D0DBB202F8013B0134082CE9D10B7A202B48
S315080014E022D0561C2E2313700B7A202B1BD001F109
S315080014F00804171D324608F010085FFA88F603E05C
S3150800150014F8013F202B0FD046B1A3F1410C5FFA26
S315080015108CFCBCF1190F9CBF2033DBB202F8013BEF
S31508001520BA42EDD100E03246CB7A2B72CC7F8B7F64
S315080015301B0443EA04630C7F23434C7F43EA0423DA
S315080015402B604C7E0B7E43EA0423AB80CC7D8B7DDF
S3150800155043EA0423EB8000231370AE6946B3EB69B4
S3150800156033B3036900240BB3028C4FF6FF739A4218
S3150800157008BF00241AD0C769388890B10024A0464D
S31508001580414601F02BFC70B1EA69013AA2420CD936
S315080015900134321902F8010C37F8020F0028EFD18E
S315080015A004E0002402E0002400E000240023335570
S315080015B0BDE8F08110B50446FFF72AFD034600286A
S315080015C054D12378032B49D16379002B46D00023C5
S315080015D0236304F1340104F50D700B46002203F869
S315080015E0012B8342FBD1552384F83232AA2384F88F
S315080015F03332522384F8343084F83530612384F842
S315080016003630412284F83720722084F8180284F88C
S31508001610190284F81A2284F81B32236984F81C32CA
S31508001620C3F3072284F81D221A0C84F81E221B0E07
S3150800163084F81F32E36884F82032C3F3072284F85B
S3150800164021221A0C84F822221B0E84F82332607891
S3150800165062690123FFF7E8F90023637160780021C6
S315080016600A46FFF745FA031C18BF0123184610BDA2
S3150800167002398369023B99423DBF8278C36A02FBFD
S3150800168001300020704700BFF8B505460C46012911
S315080016905CD9836999425BD20378022B28D0032B45
S315080016A038D0012B56D101EB5106416A01EB562180
S315080016B0FFF7EAFC002850D1C6F308032B4493F839
S315080016C034700136696A284601EB5621FFF7DCFCBF
S315080016D0002845D1C6F30806354495F8340047EA8C
S315080016E0002014F0010F14BF0009C0F30B00F8BD69
S315080016F0416A01EB1421FFF7C7FCA0BB640004F4A0
S31508001700FF742B1993F834302C4494F8350043EAC7
S315080017100020F8BD416A01EBD411FFF7B5FC28BBE0
S31508001720A40004F4FE742B1993F8360093F83720B6
S31508001730120642EA004293F8350042EA00202C4499
S3150800174094F83430184320F07040F8BD0120F8BDF5
S315080017500120F8BD4FF0FF30F8BD4FF0FF30F8BD5F
S315080017604FF0FF30F8BD4FF0FF30F8BD4FF0FF30B7
S31508001770F8BD00BF70B504460D46E18081680129B1
S3150800178038D003689A69914236D271B91A78032A11
S3150800179001D1996A49B90022E2601A89AA422DD96B
S315080017A09B6A03EB151323611BE09E783601B5424D
S315080017B010D32068FFF768FF0146B0F1FF3F1FD03E
S315080017C001281FD923689B6998421DD2AD1BADB26B
S315080017D0AE42EED9E1602068FFF74AFF00EB15102C
S315080017E0206105F00F05236803EB45133433636165
S315080017F0002070BD022070BD022070BD022070BDA1
S31508001800012070BD022070BD022070BDF8B50546E6
S315080018100C461646012998BF02237CD9836999424A
S3150800182028BF022377D20378022B40D0032B50D04F
S31508001830012B18BF02236BD101EB5107416A01EB5B
S315080018405721FFF721FC0346002861D1C7F3080397
S3150800185014F001041FBFEA1892F8342002F00F02B0
S31508001860F1B21ABF42EA0112D2B2F2B22B4483F89D
S315080018703420013701232B71696A284601EB572169
S31508001880FFF702FC0346002842D1C7F3080714B144
S31508001890C6F3071607E0EA1992F8342022F00F0279
S315080018A0C6F3032616432F4487F8346030E0416AAE
S315080018B001EB1421FFF7E8FB034648BB640004F478
S315080018C0FF742A1982F83460C6F3072682F8356051
S315080018D01EE0416A01EBD411FFF7D6FB0346B8B9FF
S315080018E0A40004F4FE742A1992F8371009062C4449
S315080018F001F070410E4384F83460C6F3072182F87C
S315080019003510310C82F83610360E82F83760FFE74C
S3150800191001222A71FFE71846F8BD00BF2DE9F041FC
S315080019200546884631B9C66876B183699E4228BF9E
S3150800193001260AE0FFF7A8FE012847D9AB699842B5
S3150800194028BF464601D24DE0012634460227013417
S31508001950AB699C4202D3012E3BD93C462846214618
S31508001960FFF792FE38B1B0F1FF3F18BF012833D018
S31508001970B442ECD132E02646284621466FF0704242
S31508001980FFF744FF0346D0F1010038BF0020B8F145
S31508001990000F08BF002028B1284641462246FFF717
S315080019A035FF03465BB9EE602B69B3F1FF3F18D0EC
S315080019B0013B2B6101236B712046BDE8F081012BA9
S315080019C014BF01204FF0FF30BDE8F0810120BDE8CB
S315080019D0F0810020BDE8F081BDE8F0810020BDE877
S315080019E0F0812046BDE8F0812DE9F84304460E460D
S315080019F0C5880135ADB2002D6AD00369002B6AD0BF
S31508001A0015F00F075BD101330361C16821B903687B
S31508001A101B89AB4262D952E000688378013B13EA1E
S31508001A2015134CD1FFF730FE8046012859D9B0F17D
S31508001A30FF3F59D020688369984539D3002E56D080
S31508001A40E168FFF76BFF8046002853D0012854D081
S31508001A50B0F1FF3F54D02068FFF7DAFA002852D1D8
S31508001A60236803F1340100231A46CA540133B3F537
S31508001A70007FFAD1266830464146FFF7F9FD306304
S31508001A8000264FF001090CE083F804902068FFF760
S31508001A90BFFA00283AD123681A6B01321A63013655
S31508001AA0F6B223689A78B242EED81A6B921B1A637A
S31508001AB0C4F80C8020684146FFF7DAFD2061E5800E
S31508001AC0236803EB4713343363610020BDE8F883CA
S31508001AD00420BDE8F8830420BDE8F8830420BDE8A7
S31508001AE0F8830220BDE8F8830120BDE8F8830420C6
S31508001AF0BDE8F8830720BDE8F8830220BDE8F8832F
S31508001B000120BDE8F8830120BDE8F8830120BDE87F
S31508001B10F88300BF2DE9F04F89B005460021FFF78D
S31508001B2029FE002840F0AC804FF0FF09C8464F4612
S31508001B3044F27471C0F60001029101F10C0204929C
S31508001B404FF6FF7A4FF0000B28682969FFF79CFAD1
S31508001B50002840F096806C692678002E00F0928066
S31508001B60E37A03F03F02E52E7FD013F0080F04D086
S31508001B700F2A18BFB8467BD101E00F2A58D1EB6966
S31508001B800193002B74D016F0400F06D094F80D90F0
S31508001B9006F0BF06EB882B8403E0B04518BFB846AD
S31508001BA066D1617B0391494518BFB84660D1237851
S31508001BB023F04003013B03EB430203EB8202059249
S31508001BC0029A02F1FF394FF001080796059E06951D
S31508001BD04546DDF8108019F8013FE2185078E35CB5
S31508001BE043EA00207DB101F01FF90546FE2E56D8BE
S31508001BF0731C0593019931F8160001F015F9854211
S31508001C004FD1059E01E050454DD1C145E3D1A846C7
S31508001C100596079E069D237813F0400F39D0B8F134
S31508001C20000F36D0059A019931F812308BB33BE094
S31508001C30B8F1000F04D12046FFF78EF9484523D0A6
S31508001C40A5F820A0AB69DA7A12F0010F08BF04F1F3
S31508001C500B0002D00BE0844218D014F8011B13F8CD
S31508001C60012B9142F7D0B84602E0B84600E0B846E4
S31508001C7028465946FFF7B8FE00283FF465AF07E047
S31508001C8016E015E0042013E0002011E000200FE024
S31508001C900EE0013E5FFA86F8DDF80C90E8E7069D4F
S31508001CA002E0069D00E0069DDDF80C90B846DFE7E9
S31508001CB009B0BDE8F08F00BF2DE9F04F87B0814627
S31508001CC088460B782F2B18BF5C2B08BF01F101083B
S31508001CD00023836098F800301F2B07D80021FFF7F0
S31508001CE049FD03460022C9F814207AE14FF0010A9B
S31508001CF044F2E06BC0F6000B44F2EC61C0F600015A
S31508001D00049144F2F462C0F60002059298F8003095
S31508001D102F2B18BF5C2B08D108F10103984613F83E
S31508001D20012B2F2A18BF5C2AF8D0D9F81C5098F82E
S31508001D3000002F2818BF1F282CD95C2800F02D81F9
S31508001D40AF1E4646544607E05C2B00F02881B2F5E4
S31508001D50807F00F041811446514601F03FF8014664
S31508001D60002800F039817F2809D8222900F034811B
S31508001D705A4612F8013F13B19842FAD12CE127F8D6
S31508001D80021F621C16F8013F18462F2B18BF1F2B7F
S31508001D90DAD801E00024524690441F2898BF04264A
S31508001DA001D90026FFE7002C00F0168104F1004354
S31508001DB0013B5A0035F813302E2B18BF202B40F064
S31508001DC0F080931C2B4407E033F8042C023B2E2AA0
S31508001DD018BF202A40F0E580013CF5D1FCE003F865
S31508001DE0011B8342FBD12B88202B18BF2E2B40F0DA
S31508001DF0E48028460023013330F8021F202918BF43
S31508001E002E29F8D0002B00F0D98046F00306D5E03D
S31508001E10013C05D10821039100220192029205E0B6
S31508001E20023A32F8021C2E29F2D1F3E75F1C35F884
S31508001E301300002861D0202808D0E31B18BF01230F
S31508001E402E2814BF002203F001021AB146F0030639
S31508001E503B46EBE7019A0399BC4218BF8A4214D362
S31508001E600B2903D146F00306029A49E00BB146F066
S31508001E700306A74243D8029A9300DBB2029323468D
S31508001E800B21039108220192D0E77F280DD9002162
S31508001E9000F0A4FF0346002800F0A08005990B4433
S31508001EA013F8800C46F0020650B101462B2807D0DD
S31508001EB0049A12F8013F002B00F087809942F8D166
S31508001EC046F003065F2010E0029A42F002020292F0
S31508001ED00BE0A0F161039BB2192B9FBF029B43F055
S31508001EE001030293203898BF80B2D9F818300199B7
S31508001EF058543B460131019198E7029A00E0029A4C
S31508001F00D9F818301978E52904BF05211970039BFB
S31508001F10082B02BF9200D2B20292029901F00C037A
S31508001F200C2B03D001F00302032A01D146F0020666
S31508001F3016F0020F0AD1029901F00302012A08BF1E
S31508001F4046F01006042B08BF46F00806D9F81830E4
S31508001F50DE724846FFF7DEFDD9F81830DA7A03460E
S31508001F6048B104283DD102F00403DBB2002B14BFAC
S31508001F700346052335E012F0040F32D1D9F81410C0
S31508001F80CB7A13F0100F06D0D9F80000FEF7D4FF6D
S31508001F90C9F80800BAE6052323E00024524690440F
S31508001FA0FFE66700EA194FF0000325F81430D9F860
S31508001FB0183003F10B00202111E700232F4437F8CE
S31508001FC0021C2E293FF426AF22E7A0F141039BB25B
S31508001FD0192B7FF679AF7CE7062302E046F0020666
S31508001FE06EE7184607B0BDE8F08F00BF2DE9F04F41
S31508001FF083B0044689464FF0FF0B5E460425D84653
S3150800200044F2747AC0F6000A0AF10C03009300271A
S3150800201070E02068FFF738F8054600286ED1626937
S315080020201378002B74D0D17AE52B18BF2E2B59D0F4
S3150800203001F03F01082914BF00200120484518BFB8
S31508002040464651D10F2943D113F0400F06D092F8D6
S315080020500DB003F0BF03E188218403E09E4218BF58
S31508002060464641D192F80DE0DE4518BF46463BD1BB
S31508002070D4F81CC0117801F03F01013901EB410584
S3150800208001EB85050AF1FF3101260193DDF800B061
S3150800209011F8013FD0184078D35C43EA002036B1E6
S315080020A0FE2D32D82CF815000646013503E04FF60A
S315080020B0FF73984229D15945EAD1019B127812F04B
S315080020C0400F1ED0FE2D98BF2CF8157019D91CE0AC
S315080020D010461EB9FEF740FF58451BD04FF6FF7352
S315080020E0238417E04646FFE720463946FFF77CFC7F
S315080020F0054618B9216900298BD15DB100232361F2
S3150800210008E0013BDEB2F346EEE7F3464646EBE768
S315080021100425F3E7284603B0BDE8F08F2DE9F04122
S315080021200446C588018C4FF6FF73994208BF2946B5
S31508002130FFF720FB0346D0B9E52701264FF0000834
S3150800214020682169FEF7A0FF034668B9626917701F
S3150800215022681671E288AA4209D220464146FFF74C
S3150800216043FC03460028EBD0042B08BF022318467D
S31508002170BDE8F0812DE9F04104460E46012998BFD5
S3150800218002212BD983699E4228BF022126D2002725
S315080021904FF0010820463146FFF776FA0546C0B1EA
S315080021A0012818D0B0F1FF3F17D0204631463A46ED
S315080021B0FFF72CFB014688B92369B3F1FF3F1EBF21
S315080021C00133236184F80580A369AB4206D92E46FC
S315080021D0E0E7002102E0022100E001210846BDE80F
S315080021E0F08100BF70B582B0054616461C460B2224
S315080021F0FEF798FE052C0BD9B21EE30343EA5404F6
S31508002200A4B232F8023F1C44A4B25388002BF4D17E
S31508002210072204F00F0101F13003392B88BF01F1C1
S315080022203703013A00A911444B702409F1D1144629
S315080022307E2102AB134403F8081C62B12B78202BCD
S315080022400BD0294600230133A34207D011F8010F0A
S315080022502028F8D102E0002300E000232020072AE6
S315080022609FBF02A9891811F8081C013288BF0146C8
S31508002270E9540133072BF2D902B070BD2DE9F04FAE
S3150800228087B004468769C66903A839460C22FEF753
S3150800229049FE9DF8173013F0010F21D00023FB7279
S315080022A0E3610125384603A932462B46FFF79AFF14
S315080022B02046FFF72FFC034620B90135ADB2642D41
S315080022C0F0D1D5E0642D08BF072000F0EF80042B7D
S315080022D018BF184640F0EA809DF81730FB72E66191
S315080022E09DF8173013F0020F08BF012716D0338860
S315080022F03BB1002301339BB236F81320002AF9D1EB
S3150800230000E0002319334EF64F42C4F6C46282FB3E
S315080023100317DB17C3EBA707BFB2FFE72046002169
S31508002320FFF728FA0346002840F0BF800025A84694
S31508002330012620682169FEF7A7FE0346002840F01B
S31508002340B48063691B78E52B18BF002B03D10135D0
S31508002350AF4201D18EE0454620463146FFF744FBA1
S3150800236003460028E5D0A0E0E188C9EB0101204634
S3150800237089B2FFF7FFF90346002840F09680A06966
S31508002380FEF7EAFD01904FF000084FF6FF7544F29C
S315080023907476C0F60006FF2720682169FEF774FEEA
S315080023A00346002840F08180D4F81CA061695FFAD2
S315080023B089FB019A4A734FF00F03CB7281F80C80A0
S315080023C081F81A8081F81B800BF1FF3303EB430079
S315080023D003EB80000122434602E070462B46013299
S315080023E0AB424ED000F1010E3AF81030B01810F892
S315080023F0010C0B5408444FEA132C80F801C0002B3B
S3150800240049D070460C2AEAD9AB4202D03AF81030C5
S315080024100BB94BF0400B81F800B023684FF001016F
S31508002420197120464146FFF7DFFA034600283CD1DA
S3150800243009F1FF391FFA89F9B9F1000FACD12DE07E
S31508002440636903F12001002203F8012B8B42FBD1BB
S315080024506069A1690B22FEF765FD6369A269D27AF4
S3150800246002F018021A73236801221A7100201DE06F
S3150800247007201BE0013F1FFA87F9B9F1000F0DD0BD
S3150800248072E706EB020E1EF801EC01F80E708E4498
S315080024908EF80170B6E70C2A9FD9BAE72068216939
S315080024A0FEF7F2FD0028CBD000E0184607B0BDE8DD
S315080024B0F08F00BF88B940F23843C2F200031B68A8
S315080024C00BB100221A7009B100230B7040F2384391
S315080024D0C2F200031960002070470B20704700BF46
S315080024E02DE9F0438FB0019115460446002800F007
S315080024F094800023036001A805A902F01E02FEF7D6
S31508002500F9FD002840F08B8005F01F0702AB0B93FE
S3150800251040F23423C2F200030C9305A80199FFF791
S31508002520CBFB0A9E034600287FD1002E78D17BE09C
S315080025305BB1042B40F0858005A8FFF79FFE47F0A6
S3150800254008070A9E034638B17BE0F37A13F0110FA9
S3150800255070D115F0040F6FD117F0080F3CD0FEF7B5
S315080025600FFCB073C0F30723F373030C3374000E28
S3150800257070740025F57235777577B577F577DDF8D8
S31508002580148040463146FEF7D7FCB576F5763575A4
S315080025907575012388F804300546E8B1D8F83090F7
S315080025A040462946FFF7E6FD0346002849D1059827
S315080025B0013DC5604946FEF767FD03460AE0F37A22
S315080025C013F0100F3AD115F0020F05D013F0010FD2
S315080025D036D101E0002B34D117F0080F18BF47F0A9
S315080025E02007059D2B6BE3612662A77128463146B5
S315080025F0FEF7A2FC2061F27FB37F1B0443EA026365
S31508002600327F1343727F43EA0223E3600020A0600F
S31508002610A0612560EB88A38014E0092012E011E090
S3150800262015F01C0F91D1CAE7062315F01C0F7FF48D
S315080026307FAFCFE7072304E0082302E0042300E086
S31508002640072318460FB0BDE8F08300BF2DE9F04F09
S3150800265083B004460F4690461E4600233360FEF7B5
S315080026602DFD002840F0BF80A37913F0800F18BF16
S31508002670022040F0BC8013F0010F08BF072000F0CD
S31508002680B680E568A368ED1AA84538BF4546002D0B
S3150800269000F0AA8004F124030193A368C3F3080297
S315080026A0002A40F08680206890F802A00AF1FF3AD6
S315080026B00AEA532A1AF0FF0A17D10BB9206902E071
S315080026C06169FEF7E1FF012805D8A37963F07F0366
S315080026D0A37102208BE0B0F1FF3F05D1A37963F027
S315080026E07F03A371012082E06061D4F80080404630
S315080026F06169FEF7BDFF814628B9A37963F07F03B8
S31508002700A371022073E0D1445FEA552B29D098F8CB
S3150800271002300BEB0A029A4288BFCAEB030B98F801
S31508002720010039464A465FFA8BF3FEF72DF928B1C0
S31508002730A37963F07F03A371012058E0A37913F00E
S31508002740400F0BD0A369C9EB0300834506D907EBF5
S31508002750402001994FF40072FEF7E4FB4FEA4B2B39
S3150800276035E0A2694A4522D0A37913F0400F10D06C
S3150800277098F8010001990123FEF756F928B1A379C3
S3150800278063F07F03A371012031E0A37923F04003AE
S31508002790A3712368587801994A460123FEF7F4F88D
S315080027A028B1A37963F07F03A37101201FE0C4F861
S315080027B01890A168C1F30801C1F5007B5D4538BFD3
S315080027C0AB462144384624315A46FEF7ABFB5F44F4
S315080027D0A3685B44A36033685B443360B5EB0B05C1
S315080027E07FF45BAF02E002E0002000E0002003B0C7
S315080027F0BDE8F08F2DE9F04F83B004460F46154625
S315080028001E4600233360FEF759FC002840F0DA80A4
S31508002810A37913F0800F18BF022040F0D48013F07C
S31508002820020F08BF072000F0CE80E368DD4280F083
S31508002830BE80002D00F0BB8004F124030193A36839
S31508002840C3F30802002A40F09580206890F802B089
S315080028500BF1FF3B0BEA532B1BF0FF0B21D13BB9C6
S31508002860236963B90021FFF759F80346206103E09D
S315080028706169FFF753F80346002B00F09880012B97
S3150800288005D1A37963F07F03A37102209BE0B3F11E
S31508002890FF3F05D1A37963F07F03A371012092E07E
S315080028A06361A37913F0400F11D023685878019912
S315080028B0A2690123FEF7B8F828B1A37963F07F036C
S315080028C0A37101207FE0A37923F04003A371D4F814
S315080028D0008040466169FEF7CBFE814628B9A37998
S315080028E063F07F03A37102206DE0D9445FEA552A9D
S315080028F029D098F802300AEB0B029A4288BFCBEB34
S31508002900030A98F8010039464A465FFA8AF3FEF741
S315080029108BF828B1A37963F07F03A371012052E0F5
S31508002920A369C9EB03018A450AD9019807EB412136
S315080029304FF40072FEF7F6FAA37923F04003A37169
S315080029404FEA4A2A28E0A3694B4511D0A268E368F2
S315080029509A420DD298F8010001994A460123FEF7DA
S3150800296013F828B1A37963F07F03A37101202AE045
S31508002970C4F81890A068C0F30800C0F5007A554559
S3150800298038BFAA462044243039465246FEF7CAFACA
S31508002990A37943F04003A3715744A3685344A36043
S315080029A0336853443360B5EB0A057FF448AFA36830
S315080029B0E268934288BFE360A37943F02003A371DA
S315080029C0002000E0FFE703B0BDE8F08F38B5044605
S315080029D0FEF774FB002849D1A37913F0200F46D0DF
S315080029E013F0400F0DD0214651F8243B5878A269C0
S315080029F00123FEF719F800283BD1A37923F04003F9
S31508002A00A3712068E169FEF73FFB002833D1256AE8
S31508002A10EB7A43F02003EB72E3682B77A3891B0A52
S31508002A206B77E389AB77E37BEB772369AB76C3F305
S31508002A300722EA761B0C2B751B0A6B75FEF7A0F9A5
S31508002A40A875C0F30723EB75030C2B76000E687682
S31508002A500023AB74EB74A37923F02003A3712368D6
S31508002A6001221A712068FEF7A5FD38BD38BD002081
S31508002A7038BD012038BD38BD10B50446FFF7A6FF9E
S31508002A80034608B900222260184610BD70B50446F0
S31508002A900D46FEF713FB002840F0BD80A37913F01E
S31508002AA0800F40F0B980E268AA4205D203F002031B
S31508002AB0DBB2002B08BF1546A2680023A360002DD1
S31508002AC000F0AC802068867876026AB1013A691E01
S31508002AD0B1FBF6F1B2FBF6F3994205D373421A40FD
S31508002AE0A260AD1A616918E02169A9B9FEF716FF57
S31508002AF00146012805D1A37963F07F03A37102205B
S31508002B0070BDB0F1FF3F18BF206105D1A37963F00E
S31508002B107F03A371012070BD6161002940D0B542D1
S31508002B202BD9A27912F0020F05D02068FEF7F6FE1F
S31508002B30014620B920E02068FEF7A6FD0146B1F15E
S31508002B40FF3F05D1A37963F07F03A371012070BD10
S31508002B50012903D922689269914205D3A37963F0C2
S31508002B607F03A371022070BD6161A2683244A2602E
S31508002B70AD1BAE42D5D300E03546A2682A44A26012
S31508002B80C5F3080272B12068FEF772FD28B9A37969
S31508002B9063F07F03A371022070BD00EB552502E0A8
S31508002BA0002500E00025A368C3F3080343B3A26920
S31508002BB0AA4225D0A37913F0400F11D0214651F827
S31508002BC0243B58780123FDF72FFF28B1A37963F03A
S31508002BD07F03A371012070BDA37923F04003A3717D
S31508002BE0214651F8243B58782A460123FDF7CCFEA6
S31508002BF028B1A37963F07F03A371012070BDA56195
S31508002C00A368E26893420BD9E360A37943F02003F3
S31508002C10A371002070BD70BD022070BD002070BD7C
S31508002C20002070BD30B58FB00EAB43F8340D0D469D
S31508002C30184605A90022FEF75DFA0446A0B902ABBC
S31508002C400B9340F23423C2F200030C9305A80199B2
S31508002C50FFF732F8044638B90A9B23B105A8294676
S31508002C60FEF712FC00E0062420460FB030BD00BF78
S31508002C7030B599B018AB43F85C0D18460FA9012278
S31508002C80FEF738FA034600284DD103AB159340F2F8
S31508002C903423C2F2000316930FA80199FFF70CF824
S31508002CA0034600283FD11499062300293BD0CC7A45
S31508002CB014F0010F18BF072335D124E0012D98BF62
S31508002CC0022330D906A80FA92422FEF72BF9089566
S31508002CD006A80221FEF74EFD034620BB06A80021E2
S31508002CE0FFF784F90346E8B1042814D01BE02DB198
S31508002CF00F982946FFF73EFA0346A0B90F98FEF744
S31508002D0059FC03460FE00F98FEF716F9054614F02E
S31508002D10100FD3D1FFE70FA8FFF700FA03460028E4
S31508002D20E5D000E00723184619B030BD2DE9F04379
S31508002D3083B081469046054600244E1E012711E0C1
S31508002D40404601A93A466B46FFF780FC009B012BDB
S31508002D500AD19DF804300D2B04D005F8013B013447
S31508002D600A2B01D0A642EBDC00232B709C4214BF31
S31508002D704846184603B0BDE8F08300BF30B583B0B7
S31508002D8004460D460A2802D10D20FFF7F7FF02A9CF
S31508002D9001F8084D28466946012201ABFFF72AFDCE
S31508002DA00198012814BF4FF0FF30012003B030BD51
S31508002DB070B505460E46007860B100243146FFF727
S31508002DC0DDFFB0F1FF3F08D0013415F8010F0028E8
S31508002DD0F4D101E0002070BD204670BD7F2821D9BE
S31508002DE041B9C7281EBF44F66412C0F60002012383
S31508002DF00AD112E0FF2814D8803844F66413C0F6C6
S31508002E00000333F81000704732F8021F814205D0DC
S31508002E1001339BB2802BF7D100E000238033D8B270
S31508002E2070470020704700BF61280CD044F28472B6
S31508002E30C0F600020021013132F8023F53B1834245
S31508002E40F9D10BB97047002144F66423C0F6000394
S31508002E5033F81100704700BF08B500F0BBFA01F05F
S31508002E6027F901F00BF900F039FB00F00FF800F034
S31508002E709FFA08BD08B500F0AFFA01F035F900F081
S31508002E806BFC00F013F800F06DFA08BD10B500F001
S31508002E9087F800F0D7FE40F20104C2F200040123CD
S31508002EA0237001F043F80023237010BD08B540F2E3
S31508002EB03C40C2F2000000F0CDFF01280BD140F2E1
S31508002EC00103C2F2000301221A7040F23C40C2F22A
S31508002ED0000000F085F840F23C40C2F2000001F024
S31508002EE06FF801280BD140F20103C2F20003002259
S31508002EF01A7040F23C40C2F2000000F071F808BDBA
S31508002F00704700BF38B505460C4640F20103C2F2C9
S31508002F1000031B78012B02D1C9B200F047FF40F22B
S31508002F200103C2F200031B781BB92846E1B201F07F
S31508002F3013F800F04DF838BD40F20103C2F2000361
S31508002F401878022806D0032806D001280CBF0820C6
S31508002F5040207047002070470020704740F2010368
S31508002F60C2F200031878022806D0032806D00128E2
S31508002F700CBF08204020704700207047002070478B
S31508002F8008B500F01BF808BD40F27C43C2F2000306
S31508002F90FE22DA7018710222A3F84420704700BF97
S31508002FA040F27C43C2F2000300221A709A6483F846
S31508002FB04320A3F844209A705A70704740F27C4325
S31508002FC0C2F200031878003018BF0120704700BF0E
S31508002FD040F27C43C2F20003002283F84320704784
S31508002FE038B504460178FF2923D100F08DFA18B9BF
S31508002FF01020FFF7C9FF96E140F27C44C2F20004B4
S315080030000023637001252570FF22E27010222271C9
S315080030106371FFF791FFA071FFF7A0FFE071FFF75B
S315080030209DFF000A20726572A5720823A4F8443031
S3150800303079E140F27C43C2F200031B78012B40F091
S315080030409081C939352900F26B81DFE811F0DB0080
S31508003050690169016501690169015901FC004201BB
S315080030602F0169016901690169016901690169013C
S3150800307069016901690169016901690169016901F2
S3150800308069016901690169016901690169016901E2
S3150800309069016901690169016901690169016901D2
S315080030A069017F00540036007300690169016901EE
S315080030B0A1006901B900BD00CE004578FFF73CFFC5
S315080030C00138854203DD2220FFF75EFF2BE140F23F
S315080030D07C45C2F20005281DA96C627800F0A2FDA5
S315080030E0FF23EB706278AB6C1344AB6463780133EF
S315080030F0A5F8443017E14578FFF71EFF01388542E9
S3150800310003DD2220FFF740FF0DE1616840F27C45B0
S31508003110C2F20005A964281D627800F083FDFF232A
S31508003120EB706278AB6C1344AB6463780133A5F833
S315080031304430F8E040F27C43C2F20003FF22DA7022
S3150800314042689A640122A3F84420ECE040F27C43EA
S31508003150C2F20003FF22DA709B6C406840B1184443
S31508003160002213F8011B0A44D2B28342F9D100E0C7
S31508003170002240F27C43C2F20003C3F80720012272
S315080031801A7100225A719A710822A3F84420CAE0DB
S3150800319040F27C43C2F20003FF22DA7044F644424E
S315080031A0C0F600029A6400221A715A719A710721B0
S315080031B0D9711A725A729A720822A3F84420B2E098
S315080031C00020FFF7E1FEAEE040F27C43C2F20003C6
S315080031D0FF22DA7000221A71597859719A71DA71D8
S315080031E01A720622A3F844209DE040F27C43C2F2FC
S315080031F0000300221A705A70FF22DA700122A3F81F
S31508003200442090E040F27C43C2F200039D6CFFF735
S3150800321093FE411E2846621C00F034FF18B931207F
S31508003220FFF7B2FE7FE040F27C44C2F20004FF23BF
S31508003230E370A56CFFF780FE013D2844A0640123D6
S31508003240A4F844306FE04578FFF776FE02388542E9
S3150800325003DD2220FFF798FE65E040F27C43C2F2C8
S315080032600003FF22DA700122A3F84420617839B9F5
S3150800327000F014FF002856D13120FFF785FE52E0F2
S3150800328040F27C43C2F20003986CA21C00F0FAFEDE
S3150800329018B93120FFF778FE45E040F27C43C2F2C8
S315080032A0000361789A6C0A449A643CE040F27C44D4
S315080032B0C2F20004FF23E370002525716571FFF74C
S315080032C03BFEA071E571257265720723A4F84430A8
S315080032D029E040F27C43C2F20003986C616800F072
S315080032E0D5FE18B93120FFF74FFE1CE040F27C43AB
S315080032F0C2F20003FF22DA700122A3F8442012E08A
S3150800330000F078FC40F27C43C2F20003FF22DA7038
S315080033100122A3F8442006E03120FFF735FE02E03B
S315080033202020FFF731FE40F27C43C2F2000393F8F7
S315080033304330012B02D11020FFF726FE40F27C43D2
S31508003340C2F20003B3F844100BB2002B09DD40F2B9
S315080033507C40C2F20000012380F843300330FFF7B7
S31508003360D1FD38BD08B5FFF70BFE01281FD000F0C8
S31508003370CBF8E0B140F2C843C2F200031B78012B38
S3150800338015D100F0C3FE40F2CC43C2F200031B681D
S3150800339003F5FA7398420AD340F2C843C2F200030F
S315080033A000221A7000F0BAF808B900F023FC08BD2C
S315080033B008B540F2C843C2F2000301221A7000F0B1
S315080033C0A5FE40F2CC43C2F200031860FFF7CAFF1D
S315080033D008BD00BF704700BF704700BF00F00F036D
S315080033E0092802D903F13700704703F1300040F28B
S315080033F00403C2F200031B6803445B7803F003036B
S31508003400022B08BF2038C0B2704700BF38B5054642
S315080034100C460009FFF7E2FF207005F00F00FFF7E2
S31508003420DDFF60700023A370204638BD30B4024625
S3150800343003464CF6CD40CCF6CC400131A0FB034305
S31508003440DB08FAD1002301F801394CF6CD45CCF654
S31508003450CC450846A5FB0243DB0803EB8304A2EB35
S315080034604402303201F801291A46002BF1D130BC4A
S31508003470704700BFF0B440F20403C2F200031F68AD
S3150800348000231C46C15C7A18527802F00302022A0D
S3150800349008BF2039C9B2A1F13002D2B2A1F13A056A
S315080034A0EDB2162A94BF00260126062D8CBF354696
S315080034B046F0010565B9092A84BFA1F13702D2B2DF
S315080034C02401E4B22244D4B20133022BDAD101E05A
S315080034D0002000E02046F0BC704700BF08B540F267
S315080034E01053C2F200030020187040F21C51C2F2B9
S315080034F00001FEF7DFFF30B144F64C40C0F600008D
S315080035007C2100F069FB08BD40F21053C2F20003AB
S315080035101878D0F1010038BF0020704708B5FFF7CA
S315080035202FFD01280FD040F21053C2F200031B787A
S315080035305BB9FCF70DFE012809D140F21053C2F21F
S315080035400003187008BD002008BD002008BD002033
S3150800355008BD00BF027840F20403C2F200031B68EC
S315080035609918497801F00301022908BF203A532A1D
S315080035700ED1407803445B7813F0040F0AD0312843
S315080035800AD032280AD0332814BF032002207047F5
S3150800359003207047032070470020704701207047BA
S315080035A070B504460230FFF765FF06460546043443
S315080035B02046FFF75FFF3044C6B2013DADB2023484
S315080035C0012DF5D82046FFF755FFF643F6B2864299
S315080035D014BF0020012070BD2DE9F04115460F46A5
S315080035E00446002918BF002807D144F64C40C0F607
S315080035F0000040F2362100F0EFFA2046FFF7AAFF56
S315080036000646032808BF002000F0A2802046FFF7E0
S31508003610C7FF002800F08C80012E29D016B1022E93
S3150800362053D088E0A01CFFF725FF8046201DFFF732
S3150800363021FF06023E60A01DFFF71CFF30443860DC
S3150800364004F10806A8F103081FFA88F84046002D79
S315080036507ED00FFA88F7002F6FDD00243046FFF77B
S3150800366009FF285502360134A4B2BC42F6DB66E0EF
S31508003670A01CFFF7FFFE8046201DFFF7FBFE060491
S315080036803E60A01DFFF7F6FE06EB00263E6004F13D
S315080036900800FFF7EFFE3044386004F10A06A8F187
S315080036A004081FFA88F84046002D51D00FFA88F70B
S315080036B0002F46DD00243046FFF7DCFE285502368B
S315080036C00134A4B2BC42F6DB3DE0A01CFFF7D2FEF3
S315080036D08046201DFFF7CEFE06063E60A01DFFF7BA
S315080036E0C9FE06EB00463E6004F10800FFF7C2FE7D
S315080036F006EB00263E6004F10A00FFF7BBFE3044E5
S31508003700386004F10C06A8F105081FFA88F8404647
S31508003710F5B10FFA88F7002F17DD00243046FFF7BA
S31508003720A9FE285502360134A4B2BC42F6DB0EE0E7
S315080037304FF6FF700CE000200AE0404608E04046DD
S3150800374006E0404604E0404602E0404600E04046C7
S3150800375000B2BDE8F08100BF70B540F21053C2F266
S3150800376000031B78002B00F03382012B3FD1FCF7B6
S3150800377017FD44F66440C0F60000FCF75BFD44F60E
S315080037808840C0F60000FCF755FDFCF703FD01462E
S31508003790BD480122FEF7A4FE48B144F6B040C0F683
S315080037A00000FCF747FD0120FCF734FD70BD44F628
S315080037B0B840C0F60000FCF73DFD44F6C040C0F630
S315080037C00000FCF737FD44F6E440C0F60000FCF7BD
S315080037D031FD40F21453C2F2000300221A605A6007
S315080037E040F21053C2F2000302221A7070BD022B77
S315080037F040F0FD8040F21C54C2F2000440F67410FA
S31508003800C2F200004FF4807104F50D72FFF78EFACC
S3150800381094F93A32002B13DA44F6B040C0F60000A9
S31508003820FCF708FD0220FCF7F5FC04F50D70FFF720
S3150800383023F940F21053C2F2000300221A7070BD39
S3150800384000B340F67411C2F20001084601F5C071D2
S315080038500022FFF7C1FE0546B0F1FF3F12D144F63C
S31508003860B040C0F60000FCF7E5FC0320FCF7D2FCEC
S315080038708548FFF701F940F21053C2F2000300220F
S315080038801A7070BD2BB2002B2CDD40F21453C2F215
S3150800389000035B686BB940F21453C2F2000340F6AA
S315080038A07412C2F20002D2F880211A602DB25D604D
S315080038B018E040F67412C2F20002D2F8801140F203
S315080038C01452C2F20002126891423EBF40F21452EC
S315080038D0C2F20002116040F21452C2F200022DB286
S315080038E02B44536040F21C53C2F20003D3F83C2227
S315080038F0D3F840329A4240F06B8163480021FFF7C3
S31508003900C5F890B144F6B040C0F60000FCF792FC4A
S315080039100420FCF77FFC5C48FFF7AEF840F2105332
S31508003920C2F2000300221A7070BD44F6B840C0F611
S315080039300000FCF77FFC44F61450C0F60000FCF7C4
S3150800394079FC40F21455C2F2000540F2D044C2F2A6
S31508003950000468682146FFF769FD2046FCF76AFC03
S3150800396044F62050C0F60000FCF764FC2E68300EC2
S315080039702146FFF74BFDC6F30740A11CFFF746FD9E
S31508003980C6F30720211DFFF741FDF0B2A11DFFF781
S315080039903DFD2046FCF74EFC44F6C450C0F6000038
S315080039A0FCF748FC2868696800F070FB90B944F693
S315080039B0B040C0F60000FCF73DFC0520FCF72AFCE9
S315080039C03148FFF759F840F21053C2F200030022BB
S315080039D01A7070BD44F6B840C0F60000FCF72AFC21
S315080039E040F21053C2F2000303221A7070BD032B73
S315080039F040F0EE8040F21C54C2F2000440F6741007
S31508003A00C2F200004FF4807104F50D72FFF78EF9CB
S31508003A1094F93A32002B13DA44F63C50C0F600000B
S31508003A20FCF708FC0220FCF7F5FB04F50D70FFF720
S31508003A3023F840F21053C2F2000300221A7070BD38
S31508003A4020B340F67412C2F20002104602F5C071A5
S31508003A5002F58072FFF7C0FD0546B0F1FF3F15D1AC
S31508003A6044F66050C0F60000FCF7E4FB0320FCF7C0
S31508003A70D1FB0548FFF700F840F21053C2F20003E5
S31508003A8000221A7070BD00BF500700202BB2002B11
S31508003A9059DD44F68450C0F60000FCF7CBFB2DB286
S31508003AA040F2D044C2F2000428462146FFF7BEFC85
S31508003AB02046FCF7BFFB44F69450C0F60000FCF71E
S31508003AC0B9FB40F67416C2F2000696F88301214641
S31508003AD0FFF79CFC96F88201A11CFFF797FC96F865
S31508003AE08101211DFFF792FC96F88001A11DFFF7C1
S31508003AF08DFC2046FCF79EFB44F6C450C0F6000039
S31508003B00FCF798FBD6F88001294606F5807200F086
S31508003B10B9FA90B944F6B040C0F60000FCF78AFB43
S31508003B200620FCF777FB2B48FEF7A6FF40F210535A
S31508003B30C2F2000300221A7070BD44F6B840C0F6FF
S31508003B400000FCF777FB40F21C53C2F20003D3F8DF
S31508003B503C22D3F840329A423AD144F6AC50C0F6E9
S31508003B600000FCF767FB00F099FA90B944F6B040FC
S31508003B70C0F60000FCF75EFB0720FCF74BFB154878
S31508003B80FEF77AFF40F21053C2F2000300221A70C1
S31508003B9070BD44F6B840C0F60000FCF74BFB44F68F
S31508003BA0C850C0F60000FCF745FB0A48FEF764FF5C
S31508003BB044F6E050C0F60000FCF73CFB40F2105318
S31508003BC0C2F2000300221A70FCF702FB00F012F89A
S31508003BD070BD00BF5007002008B540F6F823C2F2B2
S31508003BE00003186040F6FC23C2F200031960FFF7D1
S31508003BF0F3FBFCE708B500F04DFA90B1FFF780F942
S31508003C0000F06AFA00F010FD20F0604020F07F0016
S31508003C104EF60853CEF20003186000F005FD43681F
S31508003C20984708BD70B5561EB6B24AB14C1E0E442A
S31508003C30451A14F8013F2B55FFF7CEFBB442F8D1CD
S31508003C4070BD00BF2DE9F047002344F63060C0F68A
S31508003C5000004FF4FA7448F6A04113F80080C21821
S31508003C6092F801C008EB0C0202FB044291FBF2F940
S31508003C7002FB191636B94D4609F1FF3292B2B2F572
S31508003C80806F03D30233242BE7D187E04746E24609
S31508003C904FF4C843C4F2000300225A611A6842F47A
S31508003CA000421A601B6813F4004F09D04FF4C84449
S31508003CB0C4F20004FFF790FB236813F4004FF9D110
S31508003CC04FF4C843C4F200031A6822F002021A60CD
S31508003CD01A6842F001021A605B6813F0010F09D1F5
S31508003CE04FF4C844C4F20004FFF776FB636813F088
S31508003CF0010FF9D0013F0AF1FF36360546EA0747B4
S31508003D00013D3D434FF4C843C4F20003DD611A6820
S31508003D1022F001021A605B6813F0010F09D04FF414
S31508003D20C844C4F20004FFF757FB636813F0010F99
S31508003D30F9D14FF4C843C4F20003D3F8002242F085
S31508003D400102C3F80022D3F81C2222F00102C3F8AC
S31508003D501C22D3F80C2242F00102C3F80C220022DE
S31508003D60C3F84022C3F84422D3F8042222F0010201
S31508003D70C3F80422D3F8142222F00102C3F814224D
S31508003D80D3F81C2242F00102C3F81C22D3F8002201
S31508003D9022F00102C3F80022BDE8F08744F60C6061
S31508003DA0C0F60000E621FFF717FF71E738B50446AD
S31508003DB00D464FF4C843C4F200039B6813F0806FA6
S31508003DC007D144F60C60C0F6000040F22511FFF753
S31508003DD003FF4FF4C843C4F20003D3F8802102F06E
S31508003DE00102C3F88021D3F8802142F07C4242F4D4
S31508003DF00012C3F88021C3F88451E178A27812042E
S31508003E0042EA016221780A43617842EA0122C3F84C
S31508003E108821E179A279120442EA016221790A43EA
S31508003E20617942EA0122C3F88C21D3F8802142F055
S31508003E300102C3F880219B6813F0806F09D14FF403
S31508003E40C844C4F20004FFF7C7FAA36813F0806FEA
S31508003E50F9D038BD4FF4C843C4F20003DB6813F049
S31508003E60030F39D04FF4C843C4F20003D3F8B02186
S31508003E7040F26763B3EB525F18BF002023D14FF4BB
S31508003E80C843C4F20003D3F8B8210270D3F8B821A6
S31508003E90120A4270D3F8B821120C8270D3F8B821EE
S31508003EA0120EC270D3F8BC210271D3F8BC21120AD3
S31508003EB04271D3F8BC21120C8271D3F8BC311B0EA7
S31508003EC0C3710120FFE74FF4C843C4F20003DA6860
S31508003ED042F02002DA6070470020704710B54FF4B0
S31508003EE08843C4F200031B8803F080039BB2B3B176
S31508003EF04FF48843C4F2000398801B8803F08003BC
S31508003F009BB273B94FF48844C4F20004FFF764FA0D
S31508003F10238803F080039BB2002BF7D003E0002030
S31508003F2010BD012010BD012010BD00BF4FF488430D
S31508003F30C4F2000300221A819A811A829A821A838D
S31508003F4040F271221A819A8992B242F4005242F0E2
S31508003F500C029A81704700BF2DE9F04106460C46CF
S31508003F60402906D944F65460C0F600008E21FFF7B2
S31508003F7033FE2046FFF7B2FF012806D044F6546008
S31508003F80C0F600009221FFF727FE2546ACB10024B3
S31508003F9044F65467C0F600074FF09B08FFF71CFA73
S31508003FA0305DFFF79BFF012803D038464146FFF7EF
S31508003FB013FE0134A3B2AB42F0D3BDE8F08100BFD3
S31508003FC010B540F64533C2F200031B7803BB4FF425
S31508003FD08843C4F200031B8803F020039BB2002B1E
S31508003FE044D04FF48843C4F200039A8840F600335D
S31508003FF0C2F200031A7040F64533C2F200030122EA
S315080040001A7040F64433C2F200030020187010BD3F
S3150800401040F64433C2F200031A784FF48843C4F2D8
S3150800402000031B8803F020039BB20BB34FF48843AD
S31508004030C4F200039C8840F60033C2F200039918C4
S315080040404C700132D2B240F64431C2F200010A7015
S315080040501B7893420ED10849FFF7E4FD40F6453335
S31508004060C2F2000300221A70012010BD002010BD04
S31508004070002010BD002010BD010B002008B500F07F
S3150800408057F908BD08B500F061F908BD08B500F094
S3150800409085F908BD08B500F06DFA08BD08B500F049
S315080040A03DFA10B100F09AFA08BD002008BD00BF1D
S315080040B04EF21003CEF2000300221A6041F63F11B9
S315080040C0C0F2010159609A600521196040F648332B
S315080040D0C2F200031A6070474EF21003CEF20003D4
S315080040E000221A60704700BF4EF21003CEF200039A
S315080040F01B6813F4803F1FBF40F64833C2F2000323
S315080041001A68013218BF1A60704700BF08B5FFF772
S31508004110EBFF40F64833C2F20003186808BD00BF3B
S315080041204FF40053C4F202031A6942F080021A617E
S31508004130704700BFF8B507460024254644F678665A
S31508004140C0F60006FFF748F9A359BB420ED8311945
S3150800415049680B449F4209D244F67863C0F60003C7
S3150800416005EB450203EB8203187AF8BD01350C34DA
S315080041709C2CE7D1FF20F8BD2DE9F843804600685E
S31508004180FFF7D8FFFF285CD04FF40053C4F20203B0
S3150800419040F22312C4F267525A6048F6AB12CCF6C4
S315080041A0EF525A603422DA60DB6813F0010F04D04C
S315080041B0FFF7B6FF0020BDE8F8834FF40053C4F2BA
S315080041C002031A6942F001021A61002508F104097E
S315080041D04FF40054C4F20204D8F80030EF1859F826
S315080041E00560B2B2EA52E36813F0010F05D0FFF793
S315080041F0F3F8E36813F0010FF9D1330C7B80E36819
S3150800420013F0010F05D0FFF7E7F8E36813F0010F85
S31508004210F9D13B68B34204D10435B5F5007FDBD14B
S3150800422001E0002400E001244FF40053C4F2020325
S315080042301A6922F001021A61FFF772FF2046BDE8EB
S31508004240F8830020BDE8F88338B504460D4640F6E5
S315080042504C33C2F20003984209D04FF4C043C0F66B
S31508004260000399420BD0FFF787FF20B917E040F605
S315080042705054C2F20004C5F3080393B903E040F6AC
S315080042804C34C2F2000423689D420CD0204640F804
S31508004290045B29464FF40072FFF7C4FC03E00020D4
S315080042A038BD002038BD204638BD00BF2DE9F04195
S315080042B006460C4617461D464FEA51284FEA482837
S315080042C00368B3F1FF3F06D140F8048B41464FF42B
S315080042D00072FFF7A7FC3368434505D030464146D0
S315080042E0FFF7B2FF0646D0B13368E41A3444043403
S315080042F008F50078FFF770F8331DE31AB3F5007F69
S3150800430006D330464146FFF79FFF064650B1041DC7
S3150800431017F8013B04F8013B013DEBD105E000200D
S31508004320BDE8F0810020BDE8F0810120BDE8F081FC
S3150800433040F65053C2F200034FF0FF321A6040F6BF
S315080043404C33C2F200031A60704700BF70B50446CA
S315080043500D461646FFF7EEFEFF281BD0681E2044C2
S31508004360FFF7E8FEFF2817D0620A4FF4C043C0F6ED
S315080043700003B3EB422F07BF40F64C30C2F20000F1
S3150800438040F65050C2F20000214632462B46FFF74F
S315080043908DFF70BD002070BD002070BD2DE9F8436B
S315080043A004460E46FFF7C6FE0546701E2044FFF774
S315080043B0C1FE0446FF2D18BFFF2800F0AB808542DA
S315080043C000F29F80022D40F29F800F2800F29F8006
S315080043D04FF40053C4F2020340F22312C4F26752A8
S315080043E05A6048F6AB12CCF6EF525A603422DA60BD
S315080043F0DB6813F0010F04D0FFF792FE0020BDE83A
S31508004400F8834FF40053C4F202031A6942F0020219
S315080044101A6144F67869C0F600094F460026FEF789
S31508004420DBFF3B7AAB4208D144F67863C0F600035B
S3150800443006EB460253F8227005E001360C370D2EBE
S31508004440EDD14FF0FF37C8460025FEF7C5FF98F8AF
S315080044500830A34208D144F67863C0F6000305EB9A
S31508004460450253F8228006E0013508F10C080D2DA7
S31508004470EBD14FF0FF384E460025FEF7ADFF337AF5
S31508004480A34209D144F67863C0F6000305EB45025A
S3150800449003EB82035B6804E001350C360D2DECD185
S315080044A00023C7EB08084344C3F38F23E3B1013B5A
S315080044B09EB20136B60200254FF40054C4F2020437
S315080044C0EB196361236943F040032361E36813F042
S315080044D0010F05D0FEF780FFE36813F0010FF9D14D
S315080044E005F58065B542EBD14FF40053C4F20203DB
S315080044F01A6922F002021A61FFF712FE0120BDE8CE
S31508004500F8830020BDE8F8830020BDE8F883002082
S31508004510BDE8F8830020BDE8F88300BF00B583B086
S3150800452040F64C33C2F200031B68B3F1FF3F08BFE5
S3150800453001201CD040F64C33C2F2000399685A6831
S315080045401144DA6811441A6911445A6911449A697E
S315080045500A44D96953185B4202AA42F8043D46F256
S315080045605010C0F600000421FFF7F0FEFFE703B085
S315080045705DF804FB46F20402C0F600024FF4C0439D
S31508004580C0F6000310681B68184446F20803C0F614
S3150800459000031B68184446F20C03C0F600031B68A8
S315080045A0184446F21003C0F600031B68184446F286
S315080045B01403C0F600031B68184446F21803C0F635
S315080045C000031B68184446F25013C0F600031B6824
S315080045D01844D0F1010038BF0020704708B540F6EE
S315080045E04C33C2F200031B68B3F1FF3F06D040F616
S315080045F04C30C2F20000FFF7BFFD88B140F65053B9
S31508004600C2F200031B68B3F1FF3F0BD040F65050CF
S31508004610C2F20000FFF7B0FD003018BF012008BD48
S31508004620002008BD012008BD4FF4C040C0F60000B8
S31508004630704700BF08B544F61470C0F6000036216E
S31508004640FFF7CAFA08BD00BF10B572B640F20002FD
S31508004650C2F2000240F20803C2F200039A4210D2E4
S31508004660131D0E4CE41A24F00304043400231046E8
S3150800467045F24401C0F600015A581A500433A342C1
S31508004680FAD1074807494FF000028842B8BF40F8F8
S31508004690042BFADBFBF7FEFD10BD00BF0B00002064
S315080046A008000020540F00202F64656D6F70726F2C
S315080046B0675F6F6C696D65785F73746D33327031DF
S315080046C030332E73726563002F626F6F746C6F6779
S315080046D02E747874000000006D61696E2E63000008
S315080046E0222A3A3C3E3F7C7F000000002B2C3B3DB3
S315080046F05B5D0000809A90418E418F804545454913
S3150800470049498E8F9092924F994F555559999A9B30
S315080047109C9D9E9F41494F55A5A5A6A7A8A9AAABAA
S31508004720AC21AEAFB0B1B2B3B4B5B6B7B8B9BABBCF
S31508004730BCBDBEBFC0C1C2C3C4C5C6C7C8C9CACB33
S31508004740CCCDCECFD0D1D2D3D4D5D6D7D8D9DADB23
S31508004750DCDDDEDFE0E1E2E3E4E5E6E7E8E9EAEB13
S31508004760ECEDEEEFF0F1F2F3F4F5F6F7F8F9FAFB03
S31508004770FCFDFEFF01030507090E10121416181C8E
S315080047801E000000610062006300640065006600A8
S315080047906700680069006A006B006C006D006E00B7
S315080047A06F00700071007200730074007500760067
S315080047B07700780079007A00A100A200A300A5007E
S315080047C0AC00AF00E000E100E200E300E400E50031
S315080047D0E600E700E800E900EA00EB00EC00ED007F
S315080047E0EE00EF00F000F100F200F300F400F5002F
S315080047F0F600F800F900FA00FB00FC00FD00FE00D8
S31508004800FF00010103010501070109010B010D0163
S315080048100F01110113011501170119011B011D01D2
S315080048201F01210123012501270129012B012D0142
S315080048302F0131013301350137013A013C013E01AF
S31508004840400142014401460148014B014D014F0117
S31508004850510153015501570159015B015D015F0182
S31508004860610163016501670169016B016D016F01F2
S3150800487071017301750177017A017C017E0192014C
S31508004880B103B203B303B403B503B603B703B8035E
S31508004890B903BA03BB03BC03BD03BE03BF03C0030E
S315080048A0C103C303C403C503C603C703C803C903B7
S315080048B0CA0330043104320433043404350436049C
S315080048C03704380439043A043B043C043D043E04E6
S315080048D03F04400441044204430444044504460496
S315080048E04704480449044A044B044C044D044E0446
S315080048F04F045104520453045404550456045704EF
S31508004900580459045A045B045C045E045F0470216D
S3150800491071217221732174217521762177217821DD
S3150800492079217A217B217C217D217E217F2141FFEE
S3150800493042FF43FF44FF45FF46FF47FF48FF49FF45
S315080049404AFF4BFF4CFF4DFF4EFF4FFF50FF51FFF5
S3150800495052FF53FF54FF55FF56FF57FF58FF59FFA5
S315080049605AFF0000C700FC00E900E200E400E0008E
S31508004970E500E700EA00EB00E800EF00EE00EC00D7
S31508004980C400C500C900E600C600F400F600F2003F
S31508004990FB00F900FF00D600DC00A200A300A5007A
S315080049A0A7209201E100ED00F300FA00F100D10022
S315080049B0AA00BA00BF001023AC00BD00BC00A100CD
S315080049C0AB00BB0091259225932502252425612558
S315080049D06225562555256325512557255D255C25D0
S315080049E05B251025142534252C251C2500253C255A
S315080049F05E255F255A255425692566256025502597
S31508004A006C25672568256425652559255825522569
S31508004A1053256B256A2518250C25882584258C257C
S31508004A2090258025B103DF009303C003A303C303C6
S31508004A30B500C403A6039803A903B4031E22C6033C
S31508004A40B50329226122B10065226422202321238D
S31508004A50F7004822B0001922B7001A227F20B200B8
S31508004A60A025A0004100420043004400450046003E
S31508004A704700480049004A004B004C004D004E00D4
S31508004A804F00500051005200530054005500560084
S31508004A905700580059005A002100E0FFE1FFE5FFE2
S31508004AA0E2FFE3FFC000C100C200C300C400C500A6
S31508004AB0C600C700C800C900CA00CB00CC00CD009C
S31508004AC0CE00CF00D000D100D200D300D400D5004C
S31508004AD0D600D800D900DA00DB00DC00DD00DE00F5
S31508004AE07801000102010401060108010A010C010E
S31508004AF00E01100112011401160118011A011C01F8
S31508004B001E01200122012401260128012A012C0167
S31508004B102E01300132013401360139013B013D01D4
S31508004B203F0141014301450147014A014C014E013C
S31508004B30500152015401560158015A015C015E01A7
S31508004B40600162016401660168016A016C016E0117
S31508004B50700172017401760179017B017D01910171
S31508004B60910392039303940395039603970398037B
S31508004B7099039A039B039C039D039E039F03A0032B
S31508004B80A103A303A403A503A603A703A803A903D4
S31508004B90AA031004110412041304140415041604B9
S31508004BA01704180419041A041B041C041D041E0403
S31508004BB01F042004210422042304240425042604B3
S31508004BC02704280429042A042B042C042D042E0463
S31508004BD02F0401040204030404040504060407045C
S31508004BE0080409040A040B040C040E040F046021CB
S31508004BF0612162216321642165216621672168217B
S31508004C0069216A216B216C216D216E216F2121FF9B
S31508004C1022FF23FF24FF25FF26FF27FF28FF29FF62
S31508004C202AFF2BFF2CFF2DFF2EFF2FFF30FF31FF12
S31508004C3032FF33FF34FF35FF36FF37FF38FF39FFC2
S31508004C403AFF00004F70656E424C54002E2E2F2EF0
S31508004C502E2F2E2E2F536F757263652F66696C651E
S31508004C602E6300004669726D7761726520757064FF
S31508004C706174652072657175657374206465746501
S31508004C80637465640A0D00004F70656E696E67206F
S31508004C906669726D776172652066696C6520666FF4
S31508004CA0722072656164696E672E2E2E0000000000
S31508004CB04552524F520A0D004F4B0A0D0000000094
S31508004CC05374617274696E67207468652070726FB8
S31508004CD06772616D6D696E672073657175656E6360
S31508004CE0650A0D0050617273696E67206669726D98
S31508004CF0776172652066696C6520746F206F6274CF
S31508004D0061696E2065726173652073697A652E2EF6
S31508004D102E00000045726173696E6720000000006E
S31508004D202062797465732066726F6D206D656D6F8C
S31508004D307279206174203078000000005265616441
S31508004D40696E67206C696E652066726F6D2066698C
S31508004D506C652E2E2E4552524F520A0D0000000049
S31508004D60496E76616C696420636865636B73756DFB
S31508004D7020666F756E642E2E2E4552524F520A0DBE
S31508004D800000000050726F6772616D6D696E672072
S31508004D900000000020627974657320746F206D65C9
S31508004DA06D6F7279206174203078000057726974CB
S31508004DB0696E672070726F6772616D2063686563DC
S31508004DC06B73756D2E2E2E00436C6F73696E67209C
S31508004DD06669726D776172652066696C650A0D0091
S31508004DE04669726D776172652075706461746520B5
S31508004DF07375636365737366756C6C7920636F6D21
S31508004E00706C657465640A0D000000002E2E2F2E46
S31508004E102E2F2E2E2F536F757263652F41524D43D9
S31508004E204D335F53544D33322F63616E2E6300004A
S31508004E3005020602060307030803090309040A0410
S31508004E400B040C040C050D050E050F050F061006C0
S31508004E50100710082E2E2F2E2E2F2E2E2F536F753D
S31508004E607263652F41524D434D335F53544D333270
S31508004E702F756172742E6300006000080020000020
S31508004E800300000000800008002000000400000065
S31508004E9000A00008002000000500000000C000086F
S31508004EA0002000000600000000E0000800200000C6
S31508004EB007000000000001080020000008000000AC
S31508004EC00020010800200000090000000040010839
S31508004ED0002000000A000000006001080020000011
S31508004EE00B00000000800108002000000C000000F4
S31508004EF000A00108002000000D00000000C0010805
S31508004F00002000000E00000000E00108002000005C
S31508004F100F0000002E2E2F2E2E2F2E2E2F536F759C
S31508004F207263652F41524D434D335F53544D3332AF
S31508004F302F4743432F766563746F72732E630000A1
S31508004F40002020202020202020202828282828204B
S31508004F502020202020202020202020202020202043
S31508004F6020881010101010101010101010101010AB
S31508004F70100404040404040404040410101010109B
S31508004F801010414141414141010101010101010165
S31508004F9001010101010101010101010110101010B7
S31508004FA01010424242424242020202020202020237
S31508004FB0020202020202020202020202101010108B
S31508004FC020000000000000000000000000000000B3
S31508004FD000000000000000000000000000000000C3
S31508004FE000000000000000000000000000000000B3
S31508004FF000000000000000000000000000000000A3
S315080050000000000000000000000000000000000092
S315080050100000000000000000000000000000000082
S315080050200000000000000000000000000000000072
S315080050300000000000000000000000000000000062
S30908005040000000005E
S30D0800504401040000404F0008BA
S70508000000F2
